:020000021000EC
:10F800000C9446FC0C9463FC0C9463FC0C9463FC19
:10F810000C9463FC0C9463FC0C9463FC0C9463FCEC
:10F820000C9463FC0C9463FC0C9463FC0C9463FCDC
:10F830000C9463FC0C9463FC0C9463FC0C9463FCCC
:10F840000C9463FC0C9463FC0C9463FC0C9463FCBC
:10F850000C9463FC0C9463FC0C9463FC0C9463FCAC
:10F860000C9463FC0C9463FC0C9463FC0C9463FC9C
:10F870000C9463FC0C9463FC0C9463FC0C9463FC8C
:10F880000C9463FC0C9463FC0C9463FC11241FBE69
:10F89000CFEFD0E1DEBFCDBF11E0A0E0B1E0E6E800
:10F8A000FEEF01E00BBF02C007900D92A230B1073E
:10F8B000D9F712E0A2E0B1E001C01D92AC30B1076F
:10F8C000E1F70C94A7FC0C9400FC809104018130BA
:10F8D00039F45F9BFECF8CB1992787FD90950895F1
:10F8E00080E090E00895982F80910401813019F410
:10F8F0005D9BFECF9CB908950E9465FC803231F477
:10F9000084E10E9473FC80E10E9473FC0895CF9310
:10F91000C82F0E9465FC803249F484E10E9473FC88
:10F920008C2F0E9473FC80E10E9473FCCF9108959C
:10F93000282F90E0981750F430910401313019F4D9
:10F940005F9BFECF8CB19F5F9217C0F30895CFEFFE
:10F95000D0E1DEBFCDBF8091640081608093640000
:10F96000809165008E7F8093650080EA9FE001971B
:10F97000F1F7000012981A9A0A9903C081E0809367
:10F98000040180910401882379F4809164008E7FC2
:10F9900080936400809165008E7F80936500E09184
:10F9A0000201F0910301099580910401882319F463
:10F9B00081E08093040180910401813059F480E159
:10F9C00089B91092900082E08BB986E0809395000F
:10F9D00088E18AB98091640081608093640080919D
:10F9E00065008160809365000E9465FC803309F4A6
:10F9F0007AC08133E1F40E9465FCC82F8032A1F700
:10FA000084E10E9473FC81E40E9473FC86E50E94FD
:10FA100073FC82E50E9473FC8C2F0E9473FC89E4C6
:10FA20000E9473FC83E50E9473FC80E5C8C18F3F90
:10FA3000F9F40E9465FCC82F8936B1F687E50E946B
:10FA400073FC8C2F0E9473FC82E70E9473FC8C2F46
:10FA50000E9473FC8EE60E9473FC87E60E9473FC92
:10FA600086E50E9473FC81E30E9473FC8AE0AAC1D0
:10FA7000803439F40E9465FC8638A8F10E9465FC48
:10FA800032C08134A1F40E9465FC803809F445C07D
:10FA9000813811F481E09DC1823811F48FE099C161
:10FAA000893819F0883909F093C183E092C1823412
:10FAB00011F484E103C0853421F485E00E9498FCB0
:10FAC00012C0803581F0813571F0823561F0833567
:10FAD00051F0853559F40E9465FC809305010E9420
:10FAE00065FC809306010E947CFC7ECF8635B9F4CC
:10FAF0000E9465FC182F0E9465FC0E9465FCC82FBF
:10FB00000E9465FC103309F063C1CC2311F48EE12F
:10FB100060C1C13011F487E95CC182E05AC184360A
:10FB200009F0CFC00E9465FC809308020E9465FC2A
:10FB30008093070280910B028E7F80930B020E94BC
:10FB400065FC853429F480910B02816080930B025F
:10FB5000C0E0D0E08091070290910802C817D90751
:10FB600078F407E011E00E9465FCF80181938F01B1
:10FB700021968091070290910802C817D90798F33F
:10FB80000E9465FC803209F02FCF80910B0280FF2C
:10FB900026C0C0E0D0E08091070290910802C8170B
:10FBA000D90708F08CC0E7E0F1E0A0910501B09121
:10FBB00006018191082E0E9437FF809105019091E6
:10FBC000060101969093060180930501219680918C
:10FBD000070290910802C817D90738F370C08091C6
:10FBE000060187FF04C081E080930A0202C01092E0
:10FBF0000A0280910A028BBF809105019091060153
:10FC0000880F991F90930601809305018091070248
:10FC100080FF09C08091070290910802019690939D
:10FC2000080280930702F894E199FECF1127E09132
:10FC30000501F0910601C7E0D1E0809107029091A3
:10FC40000802103091F40091680001700130D9F37E
:10FC500003E000936800E8950091680001700130AE
:10FC6000D9F301E100936800E8950990199000919B
:10FC7000680001700130D9F301E000936800E89555
:10FC80001395103898F01127009168000170013029
:10FC9000D9F305E000936800E895009168000170D1
:10FCA0000130D9F301E100936800E895329602979C
:10FCB00009F0C7CF103011F00296E5CF112484E18E
:10FCC0007EC0843709F06AC00E9465FC80930802F8
:10FCD0000E9465FC809307028091050190910601C6
:10FCE00020910B0297FF02C0226001C02D7F20935C
:10FCF0000B020E9465FC20910B02853421F42160E7
:10FD000020930B020DC02E7F20930B0280910501E2
:10FD100090910601880F991F909306018093050129
:10FD20000E9465FC803209F05FCE84E10E9473FC82
:10FD3000C0E0D0E08091070290910802C817D9076F
:10FD400008F03FC080910B0280FF08C0A091050120
:10FD5000B09106010E942FFF802D13C08695E0917F
:10FD60000501F091060180FD02C084910AC0CF0117
:10FD7000AA27BB2780509040AF4FBF4FABBFFC01BD
:10FD800087910E9473FC8091050190910601019674
:10FD900090930601809305012196CCCF8537A9F475
:10FDA0000E9465FC803209F01FCE84E10E9473FC42
:10FDB0008EE10E9473FC87E90E9473FC82E00E943E
:10FDC00073FC80E10E9473FC0FCE863709F00CCEE5
:10FDD00080E00E9487FC08CE1F93CF930E9465FCB1
:10FDE000C82F0E9473FC0E9465FC182F0E9473FCB0
:10FDF000C13614F0C75503C0C0330CF0C0531136E0
:10FE000014F0175503C010330CF01053C295C07F87
:10FE1000C10F8C2F992787FD9095CF911F91089541
:10FE2000CF93282F992787FD9095807F907044E08D
:10FE3000959587954A95E1F78A3014F0895A01C063
:10FE4000805DC22FCF70CA3014F0C95A01C0C05DA6
:10FE50000E9473FC8C2F0E9473FCCF910895E1994E
:10FE6000FECFBFBBAEBBE09A11960DB20895E199EB
:10FE7000FECFBFBBAEBB0DBA11960FB6F894E29A97
:06FE8000E19A0FBE089597
:02FE86008000FA
:040000031000F800F1
:00000001FF
